:020000040000FA
:06000000FE300C303A282E
:08000800A000030EA100831209
:10001000AA1503140B19031000308100A30DA40DC1
:10002000A50DA90B1C282A162508A8002408A7003E
:100030002308A6001930A9008B100B11210E830094
:06004000A00E200E0900D5
:0C007400203084008001840A80300402E7
:10008000031C3C281F30CE000130CA00CB00B20058
:100090008030CD000E30F5003230D70083161F308F
:1000A0008505003086050B308705831285018601A2
:1000B0008701103083168E008312703083168F00F4
:1000C00083120030031799000313003003179A00BE
:1000D00003130C30970000309F00003083169F0000
:1000E0008312183003179E000313003003179F007C
:1000F0000313803083168100831211309000043086
:1001000092007F30831692008312003095000030F9
:1001100083169400831223309400A630831698002F
:100120008312003083169B00831210309800193020
:10013000831699008312003083168C0083120030DE
:1001400083168D00831200308B008B130030031751
:100150008D0083168C130C1483120C080313F1000A
:100160000D16C32381018E018F010B118B100B1013
:100170008C018D010D168B17F02159219522F2204B
:10018000651AF920E51AF4202A1AFE208F080319AF
:10019000BE288F01E51A0717651A07150025651A8D
:1001A000F920E51AF4209B238C2324227E22651A51
:1001B000F920E51AF4204F18B421651AF920E51A40
:1001C000F42068214F18BE28AA19EC28CC0BBE28B1
:1001D000AA1AF0281930A900AA110C30CC00BE28A8
:1001E0005121BE28640008006B080E020318071393
:1001F00008006B080E020318071108002A12C1300C
:100200002802031D0A292708BB002608BA0070230C
:10021000C3234C29280827062602031D0800F730AF
:100220002802031D16292708C0004C29A1302802E6
:10023000031D1D292708F0004C29A2302802031DA8
:1002400024292708C2004C29A7302802031D35297C
:100250002A10A71B2A1427087F39EA002A1CEA0162
:100260002B142A1C2B10AB154C29C2302802031D5D
:100270004C292708C40064000D1E3C298B13440838
:1002800003178D0083168C130C1483120C080313B0
:10029000C5008B17CE164C29AA16AA110A30CC001D
:1002A00008004F144F150B12831605118312051504
:1002B00008004F10CF101930A900AA12AA110A3055
:1002C000CC008316051583128B100B110B1608003A
:1002D000E61C0800B20A0A303202031D72290630F9
:1002E000930008000E303202031D79293008930074
:1002F000080032303202031DA429350836020319E2
:10030000922903188B290230B502350836023608C7
:100310000318B50092290A30B507360835023608A9
:100320000318B500B1013518B117B51831173519D3
:10033000B116B5193116351AB115B51A3115351B67
:10034000B11424309300080036303202031DAB296B
:10035000310893000800FA303202031D08002D30E6
:10036000B200AA1CB20108004F19C129C9030F30FD
:100370004905031D0800C9080319C1290515C90E3F
:10038000080005114F11CF1859294B184608CB18F2
:1003900047084B1948084D05031DD1294430C900B1
:1003A000D4291130C900D4290310CD0C0318D92940
:1003B00008008030CD000310CB0DCB19E0290800D8
:1003C0000130CB001030CE1ACA000310CA0D03183A
:1003D0004A144A084E050319E029F021CF140800F9
:1003E000C601C701C8014A1CFA297730C600410876
:1003F000C700202ACA1C012A6630C6004308C7006D
:10040000202A4A1D082A5530C6007108C700202A34
:10041000CA1D0F2A4430C6007608C700202A4A1E8B
:10042000162A3330C6007808C700202ACA1E0800E2
:100430002130C6004408C7004508C800CE12080095
:1004400046084706C8000800051CB70A0518B70388
:100450003708031941120319B70AFF30370203198D
:1004600041160319B703851CB80A8518B803380864
:100470000319C1110319B80AFF3038020319C11555
:100480000319B803851DB90A8519B9033908031979
:1004900041110319B90AFF30390203194115031933
:1004A000B90340188616401C8612C219AC23C21923
:1004B0005D2A2A1BAC232A1F0712E619642AC01CD6
:1004C0008613C0188617682AC01C8617C0188613A2
:1004D000401F6513411C6F2A401B6F2AE5177108E6
:1004E000C11800306619F100C3187D2A2B1C7D2A23
:1004F000053078024310031C43140800E008031D74
:100500000800421C301342183017330842060239E3
:100510000319912A3016C21CB310C218B314B401C7
:100520000800B40B080030120800EA0803199F2ADB
:10053000AB18A72A6A0895002A18A12A0800950175
:10054000080006162B14AB10421AAB1408002B1D22
:1005500008002B11D518E32AD70BBE283230D7005C
:10056000D514AB19BB226A0895002A1C0800AB10F1
:10057000421AAB140800AB112130C01C013E031716
:100580008D0083168C130C1483120C080313D800EF
:100590008B17203003178D0083168C130C148312D5
:1005A0000C080313DC008B1758085C07D9005C07A4
:1005B000DA005C07DB006A087F3CDD000310DD0C1D
:1005C0000310DD0C080058087802031CF52A5908AE
:1005D0007802031CF72A5A087802031CF92A5B08E0
:1005E0007802031CFB2AD40AFD2AD00AFD2AD10A6C
:1005F000FD2AD20AFD2AD30AFD2A500851045204CA
:1006000053045404103903190800D601501AD614A3
:10061000511A5615521AD615531A5616541AD6167A
:10062000D001D101D201D301D401D5103230D7008D
:100630006A08ED005D075619ED005D07D619ED005B
:100640005D07561AED005D07D61AED006D0895009E
:1006500008003E1C08003E101030BB003D08BA00E8
:10066000702308000030BB007108BA007023080036
:10067000F10A720A71020318F1000800F103720A0C
:10068000F11BF107080064000D1E442B8B1306308C
:1006900003178D0083168C130C1483120C0803139C
:1006A0008B17401D3030F200F203701B6D2B700869
:1006B00071020318652B0319652B71087002C018AD
:1006C0007202C018013EF300080070087102C01CDD
:1006D0007202C01C013EF3000800FA30F30008006B
:1006E0000D123B08831203178D00831203133A087F
:1006F000831203178C00831603178C130C158B13AE
:100700008B1B7F2B55308D00AA308D008C148B17DE
:100710000C11831203130800F50B982B0E30F50013
:100720009F147603F7009F18932B2A151E08F600D6
:100730008D309F0008009F149F189C2B2B158B1346
:1007400083161E0883128B17F8001E08C310031DA2
:10075000C31411309F000800AE132E13AE0B080017
:10076000AD0A03302D02031C080007121E302F1C97
:100770000A302D02031C0800AF0A0130E61AAF0050
:100780000716AD01080064000D1EC42B8B138B1BD4
:10079000C62B083003178D0083168C130C1483129C
:1007A0000C080313E6008B1708000708403A87007F
:1007B00008000708043A870008000708103A870075
:1007C00008000608103A860008000608203A86004D
:0A07D00008000608803A86000800C1
:100A0000123060020318E00105308A006008820796
:100A10001A2D2E2DAB2DC32DCF2DE82D0B2E1F2ED5
:100A2000502E8E2ECB2EF42E042F1C2F282F412F2C
:100A3000572F5B2F07170711FB01FC01EB01E51393
:100A400041102923651B0800401F08006517432338
:100A5000F308031908000130E0000800AB1041144E
:100A6000B0172A17C31143138B13053003178D00DA
:100A700083168C130C1483120C080313EC008B17D1
:100A80008B13033003178D0083168C130C14831201
:100A90000C080313F9008B178B13043003178D0018
:100AA00083168C130C1483120C080313FA008B1793
:100AB0008B130C3003178D0083168C130C148312C8
:100AC0000C080313FD008B178B130D3003178D00DB
:100AD00083168C130C1483120C080313FE008B175F
:100AE0008B130E3003178D0083168C130C14831296
:100AF0000C080313FF008B178B131B3003178D009B
:100B000083168C130C1483120C080313E4008B1748
:100B10000130C01C013E8B1303178D0083168C130C
:100B20000C1483120C080313EF008B171130C01C38
:100B3000013E8B1303178D0083168C130C14831244
:100B40000C080313EE008B176C08E100FF30EB007C
:100B50000230E0000800E516E10B08006C08E10037
:100B6000EB0B0800E5128B13133003178D0083166F
:100B70008C130C1483120C080313E1008B17E20191
:100B80000330E000080007130711E20B0800E10B37
:100B900008006C08E100EB010430E0000800651675
:100BA000E10B08006C08E100EB0F0800EB03651295
:100BB0008B13143003178D0083168C130C148312BF
:100BC0000C080313E1008B17E2010530E000080078
:100BD00007130715E61CF72DE1080319F72DE61F8B
:100BE0003016E61B3017E20B0800E10B0800E61F89
:100BF0003012E61B30138B13163003178D0083164B
:100C00008C130C1483120C080313E1008B17E20100
:100C10000630E0000800E20B0800E10B08008B132F
:100C2000183003178D0083168C130C1483120C08D4
:100C30000313E1008B17E2010730E00008000616FD
:100C4000AB156E08EA00AB14661CAB10E514AA14D1
:100C50001430B6002B14E20B0800E10B0800013041
:100C6000E51BF300AB1001307302031D402E6E082C
:100C7000EA00AB14661CAB10E510AA141430B600E1
:100C80008B13193003178D0083168C130C148312E9
:100C90000C080313E1008B17E2010830E0000800A4
:100CA0003C30B60068277908760203185C2E7F086E
:100CB000FC02031C612E08007F08FC0703187D2E30
:100CC0000800FC010130E51BF300AB10013073029A
:100CD000031D732E6E08EA00AB14661CAB10E51002
:100CE000AA141430B600E20B0800E10B0800C3158B
:100CF000F3012A131130E0000800FC018B131A30B5
:100D000003178D0083168C130C1483120C08031325
:100D1000E1008B17E2010930E000080068277A083B
:100D20007602031C982E7F08FC02031C9D2E0800EF
:100D30007F08FC070318A72E0800FC01E20B08003F
:100D4000E10B08004317F3011130E0000800C01C5C
:100D50003823C0183E23F31BBB2EF30BBB2E6E08AB
:100D6000EA00AB14661CAB10E5101430B6000A3074
:100D7000E000FB0108008B13193003178D00831668
:100D80008C130C1483120C080313E1008B17E2017F
:100D90000830E00008002A1D08002A1176087702B2
:100DA000031CD72E7D08FB02031CDC2E08007E08E6
:100DB000FB070318DE2E0800FB010800FB01871269
:100DC000EA012B10AB10B0138B13173003178D00F3
:100DD00083168C130C1483120C080313E1008B1779
:100DE000E2010B30E0000800B601B501AA10322381
:100DF0000612E20B0800E10B08006C08E100FF306E
:100E0000EB000C30E00008006516E10B08006C08F0
:100E1000E100EB0B080065128B13133003178D00F4
:100E200083168C130C1483120C080313E1008B1728
:100E3000E2010D30E000080007130711E20B080083
:100E4000E10B08006C08E100EB010E30E000080047
:100E5000E516E10B08006C08E100EB0F0800EB035E
:100E6000E5128B13153003178D0083168C130C14A9
:100E700083120C080313E1008B17E2010F30E0002E
:100E8000080007170711E61C502FE1080319502F1F
:100E9000661F3016661B3017E20B0800E10B0800D6
:100EA000661F3012661B30131030E00008002A1352
:100EB0000030E00008002A13B601B501AA10B013F3
:100EC0008712EA012B10AB1006120030E000080078
:100ED000E51C0800E40B08008B131B3003178D0082
:100EE00083168C130C1483120C080313E4008B1765
:0E0EF000EA0A6F086A02031D0800E5100800F8
:084000000B00000002000000AB
:02400E00CC03E1
:1042000000007E007E00AA0096000A001800FF0051
:104210008700FF00FF00FF0041002E001400FF0098
:1042200000003200320002001400150016003700B2
:104230000600190080005A00FF00FF00FF00FF0089
:10424000050040004000FF00FF00FF00FF00FF00EE
:10425000FF00FF00FF00FF00FF00FF00FF00FF0066
:10426000FF00FF00FF00FF00FF00FF00FF00FF0056
:10427000FF00FF00FF00FF00FF00FF00FF00FF0046
:10428000FF00FF00FF00FF00FF00FF00FF00FF0036
:10429000FF00FF00FF00FF00FF00FF00FF00FF0026
:1042A000FF00FF00FF00FF00FF00FF00FF00FF0016
:1042B000FF00FF00FF00FF00FF00FF00FF00FF0006
:1042C000FF00FF00FF00FF00FF00FF00FF00FF00F6
:1042D000FF00FF00FF00FF00FF00FF00FF00FF00E6
:1042E000FF00FF00FF00FF00FF00FF00FF00FF00D6
:1042F000FF00FF00FF00FF00FF00FF0000002000A4
:00000001FF
